:020000040000FA
:0800000000008A110A124529D3
:06000A0083120313A301A1
:10001000A40122212C21F5308600831286011421AF
:1000200083120313AE00013A031D0F28102183121F
:100030000313A30023082B3A0319732823082D3A2E
:1000400003196C282308303A03196A282308313A27
:1000500003195B282308323A03195E282308333A30
:10006000031961282308343A031964282308353A10
:10007000031967282308563A0319AD282308613A63
:10008000031980282308623A0319B4282308693A1F
:100090000319BD2823086F3A031986282308703AEC
:1000A00003198B282308713A03197A282308763A12
:1000B00003199028C028AA30A400C328B430A40093
:1000C000C328D230A400C328E630A400C328FF30E0
:1000D000A400C328A401C328A0302402031CC32801
:1000E000FB30A407C328FB3024020318C3280530C3
:1000F000A407C328F53083120313860586150F283D
:10010000F53083120313860586140F280A308312F4
:10011000031386040F28F5308312031386050F2876
:100120000A2183120313AE00A0000A2183120313D5
:10013000AE00A1000A2183120313AE00A200200822
:10014000AE002108AF002208FE002F08FF002E0895
:10015000CF20A4002E30FC20C3280A2183120313D1
:10016000A4002E30FC20C3280A218312031395001B
:100170000A219B002E30FC200F284930FC200F283C
:1001800083120313A401240883120313950083121E
:1001900003132408831203139B000F280800831203
:1001A0000313AB007F08AC007E08AD00D030AB0776
:1001B000D030AC07D030AD076430FF002B08EB2007
:1001C000AB000A30FF002C08EB20AC00AB072D0879
:1001D000AB072B08080083120313A7007F08A800B1
:1001E000A901AA0127082A020318FA282808A90742
:1001F000AA0AF2282908080083120313A600831212
:1002000003130C1EFF288312031326088312031303
:1002100099000800831203138C1E0A291A0808008B
:10022000831203131A08080083120313A501831213
:1002300003138C1E1E2983120313A50A83120313B2
:100240002508080081308316031399002430980094
:100250009030831298000800083083160313810041
:100260008B170B178312920112153C3097009501E2
:100270000F3097053C309D009B010F309D05FF30EE
:1002800083169200F930870508008A110A120528A2
:00000001FF
